:020000040000FA
:060000007CEF01F012008C
:02002A000000D4
:04002C00260EE66E48
:10003000E66A3C0EE66EFEEC00F0E552E552E55253
:100040001200D9CFE6FFE1CFD9FFACA2FED7FE0E5A
:10005000DBCFE6FF65EC01F0E552E552E7CFD9FFD3
:100060001200C00EE66E080EE66E32EC01F0E552AC
:10007000E5520E0EC86E1200C5801200C584120033
:10008000D9CFE6FFE1CFD9FFC750040B01E0010E45
:10009000026E1F0EC514021001E0F6D7FE0EDBCF74
:1000A000E6FF4DEC01F0E552E552E7CFD9FF120033
:1000B000610EE66EC6DFE552C750040B01E0010E8B
:1000C000026E1F0EC514021001E0F6D7620EE66E36
:1000D000B8DFE552F70E9E149E6E080EC510C56E71
:1000E0009EA6FED7630EE66EACDFE552F70E9E14B9
:1000F0009E6EC95000D01200D9CFE6FFE1CFD9FFE4
:10010000F70E9E149E6EFE0EDB5004E0200EC5100E
:10011000C56E03D0DF0EC514C56E100EC510C56EBA
:100120009EA6FED7E552E7CFD9FF12007FDF410E32
:10013000E66E87DFE55295DF00016B6B9DDF900E69
:10014000E66E9EDFE552400EE66E9ADFE5526AC02B
:0E015000E6FF96DFE55200016A2BF9D7120098
:02015E002A0E67
:10016000F66E000EF76E000EF86E00010900F550F5
:10017000656F0900F550666F03E1656701D03DD0FA
:100180000900F550606F0900F550616F0900F550E6
:10019000626F09000900F550E96E0900F550EA6E3A
:1001A000090009000900F550636F0900F550646FFC
:1001B00009000900F6CF67F0F7CF68F0F8CF69F0D3
:1001C00060C0F6FF61C0F7FF62C0F8FF0001635333
:1001D00002E1645307E00900F550EE6E6307F8E2B0
:1001E0006407F9D767C0F6FF68C0F7FF69C0F8FF7A
:0C01F00000016507000E665BBFD712001F
:0401FC00D9CFE6FF72
:10020000DACFE6FFE1CFD9FFE2CFDAFFAC6AAB6A23
:10021000FD0EDBB0AC88DBA202D0AC8CAB8CDBB4C7
:10022000AC8EDBA602D0AB8801D0AB8ADBA802D0B3
:10023000AC8401D0AC949E98DBAC02D09D8A01D0F6
:100240009D9A9E9ADBAE02D09D8801D09D98FB0EB0
:10025000DB50AF6EAC8AAB8EE552E5CFDAFFE7CF6D
:04026000D9FF1200B0
:0C026400D9CFE6FFDACFE6FFE1CFD9FFEB
:10027000E2CFDAFF3F0EC716C66AC56AFD0EDB5035
:10028000C612FC0EDB50C71293829380C68AE552D9
:0A029000E5CFDAFFE7CFD9FF120037
:06029A00D9CFE6FFDACF28
:1002A000E6FFE1CFD9FFE2CFDAFFFD0EDB50C96EEA
:1002B000C6AE02D0FF0E03D0C7B0FED7000EE55287
:0A02C000E5CFDAFFE7CFD9FF120007
:0602CA00D9CFE6FFDACFF8
:1002D000E6FFE1CFD9FFE2CFDAFFACAC04D0AC90BF
:1002E00000016DB3AC80FD0EDB50AD6EE552E5CF85
:0802F000DAFFE7CFD9FF12008D
:0802F80013EE00F023EE00F00C
:10030000F86A019CAFEC00F096EC00F0FDD712000B
:020000040030CA
:0E000000000C1F1E008381000FC00FE00F4098
:00000001FF
